:100000001DEF1FF00000000018EF1EF000000000C0
:0C0010000000000000000000E5EF1EF002
:10001C000B820BAE18EF00F00368026801680068F1
:08002C000A360232FF0E120039
:0E003400026A016A006A086A036A000E12007E
:100042000B840BAE2CEF00F0010E036E026A016A04
:0A005200006A0A360232FF0E1200A7
:08005C000AAE029E000E120024
:100064006DB409D01F0E6B14016E0150000A03E138
:0A007400010E006E01D0006A1200B8
:10007E000CB081EF00F00CA227EF01F00E6A000E1B
:10008E00026498EF00F0F00E0214D8A463EF00F0B3
:10009E00023A01380F0B02260138F00B016E0038C0
:1000AE000F0B01260038F00B006E08380F0B0026E0
:1000BE000838F00B086E0E84D89002BE7CEF00F06C
:1000CE0008360036013602360E2A02BE7CEF00F0EC
:1000DE0008360036013602360E2A02BE7CEF00F0DC
:1000EE0008360036013602360E2A0E5003641DEF16
:1000FE0001F0035E0BBC08AE22EF01F0D880800E3B
:10010E0008640030000E002201220222D8A022EF45
:10011E0001F0023201320032034A27EF01F022EFE2
:10012E0001F001C002F000C001F008C000F0086A42
:10013E00000E0E860264CFEF00F0F00E0214D8A46B
:10014E00B7EF00F0023A01380F0B02260138F00B20
:10015E00016E00380F0B01260038F00B006E0E8476
:10016E00D89002BE7CEF00F00036013602360E2A21
:10017E0002BE7CEF00F00036013602360E2A02BEB9
:10018E007CEF00F00036013602360E2A7CEF00F0CE
:10019E0001C002F000C001F0006A000E0E960E883B
:1001AE000264FCEF00F0F00E0214D8A4E7EF00F0AA
:1001BE00023A01380F0B02260138F00B016E0E8445
:1001CE00D89002BE7CEF00F0013602360E2A02BE37
:1001DE007CEF00F0013602360E2A02BE7CEF00F0F4
:1001EE00013602360E2A7CEF00F001C002F0016AE1
:1001FE00000E0E8602642CEF01F0F00E0214D8A44D
:10020E000BEF01F0023A0E84D89002BE7CEF00F0A4
:10021E0002360E2A02BE7CEF00F002360E2A02BE15
:10022E007CEF00F002360E2A7CEF00F0010E0C6E11
:10023E0001DF2FEF01F0020E0C6E09DF2FEF01F040
:10024E00040E0C6EE4DE2FEF01F0080E0C6EEBDEEA
:02025E0012008C
:100260000A6A0350D8A40A800750D8A40A820A5008
:10027000D8B493EF01F0030AD8B44CEF01F00AB000
:1002800047EF01F006AE91EF01F08FEF01F002AE03
:100290008FEF01F091EF01F00250800B0A6E029E89
:1002A0000650800B069E0A18D8B45DEF01F00A5084
:1002B000D8B48FEF01F091EF01F00750035CD8B490
:1002C00067EF01F0D8A083EF01F089EF01F006504D
:1002D000025CD8B471EF01F0D8A083EF01F089EF90
:1002E00001F00550015CD8B47BEF01F0D8A083EF9A
:1002F00001F089EF01F00450005CD8B493EF01F0F5
:10030000D8B089EF01F00A52D8B491EF01F08FEF25
:1003100001F00A52D8B48FEF01F091EF01F0D880CC
:0E0320001200D8901200D880D884120012006B
:10032E00086A096A000E076203641CEF02F00250AD
:10033E0006180A6E075003267E0ED8A0ADEF01F008
:10034E00035ED8B020EF02F0B1EF01F0035ED8A04B
:10035E0024EF02F0028E068E02C00EF001C00BF0EA
:10036E0000C00DF000500402F4CF0CF00150050255
:10037E00F4CF00F0F3CF08F00402F3500C26F45043
:10038E000822000E00220D500502F3500C26F450E8
:10039E000822000E002202500402F3500826F450E8
:1003AE00002202500502016A000E0122F3500026BF
:1003BE00F45001220D500602F3500826F45000228C
:1003CE00026A000E012202220B500602F350002692
:1003DE00F4500122000E02220E500602F3500126A6
:1003EE00F450022202BE04EF02F008360036013647
:1003FE0002360306D8B424EF02F017EF02F0D880CD
:10040E00800E08640030000E002201220222D8A0C5
:10041E0017EF02F0023201320032034A20EF02F0EF
:10042E000AAE029E000E26EF02F0010EFCDD26EF54
:10043E0002F0020EECDD26EF02F0040EFBDD1200E0
:10044E000C6A0E6A0250D8A440EF02F001C002F00E
:10045E0000C001F0006A0E860250D8A440EF02F0F0
:10046E0001C002F0016A0E960E880250D8B452EF07
:10047E0002F00E50035ED8A4D8A057EF02F0D89029
:10048E0002BE5CEF02F0003601360236032E47EF55
:10049E0002F057EF02F0010E0C6EC5DD5FEF02F0B9
:1004AE00020E0C6EC7DD5FEF02F0040E0C6ECFDD98
:0204BE0012002A
:1004C000025006180E6E086A096A0B6A0350076428
:1004D00053EF03F006500A6E068E028E03500B6E29
:1004E0000750036E000E0B64A3EF02F00B50075E83
:1004F000D8B444EF03F0070E076412EF03F0075E71
:1005000000C008F001C000F002C001F0026A074E0E
:1005100044EF03F00764E7EF02F0075E00C008F065
:1005200001C000F0016A074E44EF03F00764C5EF15
:1005300002F0075E00C008F0006A074E44EF03F0C7
:100540000764ACEF02F00AC002F005C001F004C07D
:1005500000F0086A70EF04F0030E0764B7EF02F0D2
:10056000075E08380F0B086E074E44EF03F0D89073
:100570000832074E44EF03F0D8900832074E44EF9C
:1005800003F0D890083244EF03F0030E0764D6EF6F
:1005900002F0075E08380F0B086E0038F00B0826D3
:1005A00000380F0B006E074E44EF03F0D890003276
:1005B0000832074E44EF03F0D89000320832074E5D
:1005C00044EF03F0D8900032083244EF03F0030EFA
:1005D0000764FEEF02F0075E08380F0B086E003864
:1005E000F00B082600380F0B006E0138F00B0026C8
:1005F00001380F0B016E074E44EF03F0D890013223
:1006000000320832074E44EF03F0D8900132003236
:100610000832074E44EF03F0D8900132003208321E
:1006200044EF03F0030E07642FEF03F0075E083872
:100630000F0B086E0038F00B082600380F0B006E09
:100640000138F00B002601380F0B016E0238F00B59
:10065000012602380F0B026E074E44EF03F0D890CC
:100660000232013200320832074E44EF03F0D890D4
:100670000232013200320832074E44EF03F0D890C4
:100680000232013200320832096A000E0EAE38EF33
:1006900004F0081E001E011E021E082A002201226C
:1006A000022238EF04F00750D8A459EF03F070EF9E
:1006B00004F0096A02C00AF0028E068E0750035C3D
:1006C000076ED8B42BEF04F0070E0764F9EF03F0C0
:1006D000075E0450096E0550046E0650056E066AEA
:1006E000074E2BEF04F0070E0764CEEF03F0075E12
:1006F0000450096E0550046E056A074E2BEF04F096
:10070000070E0764ACEF03F0075E0450096E046A3D
:10071000074E2BEF04F0070E076493EF03F00AC0B7
:1007200002F070EF04F0030E07649EEF03F0075E23
:1007300009380F0B096E074E2BEF04F0D8900932E1
:10074000074E2BEF04F0D8900932074E2BEF04F040
:10075000D89009322BEF04F0030E0764BDEF03F0CD
:10076000075E09380F0B096E0438F00B09260438B0
:100770000F0B046E074E2BEF04F0D89004320932B1
:10078000074E2BEF04F0D89004320932074E2BEFBE
:1007900004F0D890043209322BEF04F0030E076402
:1007A000E5EF03F0075E09380F0B096E0438F00B14
:1007B000092604380F0B046E0538F00B04260538A3
:1007C0000F0B056E074E2BEF04F0D8900532043264
:1007D0000932074E2BEF04F0D8900532043209326B
:1007E000074E2BEF04F0D8900532043209322BEF7C
:1007F00004F0030E076416EF04F0075E09380F0BD0
:10080000096E0438F00B092604380F0B046E053806
:10081000F00B042605380F0B056E0638F00B052685
:1008200006380F0B066E074E2BEF04F0D8900632F9
:10083000053204320932074E2BEF04F0D89006320D
:10084000053204320932074E2BEF04F0D8900632FD
:10085000053204320932086A000E0EAE38EF04F099
:10086000091E041E051E061E092A04220522062250
:100870000950082604500022055001220650022289
:100880000EBE4FEF04F0D8A05EEF04F0023201324A
:1008900000320832033E5EEF04F06AEF04F0D8B095
:1008A00064EF04F0000E081E001E011E021E082A3E
:1008B0000022012202220A7E64EF04F0010E0C6E77
:1008C0003FEC00F072EF04F0020E0C6E3FEC00F013
:1008D00072EF04F0040E0C6E0EEC00F072EF04F0F8
:0608E000000E0C6E120078
:1008E6000B800BAE7FEF04F0026A0AAEFF0E026EBB
:0C08F600016E006E0A360232FF0E120086
:080902000B6A0B86FF0E1200C8
:10090A0003500718D8A499EF04F002500618D8A487
:10091A0099EF04F001500518D8A499EF04F000509B
:0E092A000418D8B4D8841200D8941200120019
:100938000B6A0A6A096A00500402F4CF09F0F3CF7F
:1009480008F001500502F4CF0BF0F3CF0AF0005085
:100958000502F3500926F4500A22E86A0B220150D6
:100968000402F3500926F4500A22E86A0B2208C050
:1009780000F009C001F00AC002F00BC003F0120039
:1009880007016651390806E3300E665D03E3010E80
:08099800006E01D0006A12009C
:1009A0000134083609360450085E0550D8A0053CCD
:1009B000095E003601360F0E0C6E0134083609361A
:1009C000045000A006D0085E0550D8A0053C095E82
:1009D00005D008260550D8B0053C0926003601365A
:1009E0000C2EEBD700B006D0045008260550D8B026
:0809F000053C0926000012007D
:1009F800086A080E0C6E003408360450085ED8B039
:0E0A080002D00826D89000360C2EF5D712002A
:100A16000050086E0150006E0250016E0350026EC7
:100A2600036A0B6A0C6A9E0E036E0A6A02AE28EF10
:100A360005F0081E001E011E021E082AD8B4002A50
:100A4600D8B4012AD8B4022A0A8E020E0C6E3FECE4
:040A560000F012009A
:100A5A00220E0C6E086A096A0A6A0B6A0C06D8B476
:100A6A001FD0D8900B320A320932083203320232CE
:100A7A0001320032D8A0F2D70C06D8B409D00450FB
:100A8A0008260550092206500A2207500B22EAD7E7
:100A9A00045008260550092206500A2207500B2244
:020AAA00120038
:100AAC0007016651200A09E066510D0804E3090E9E
:100ABC00665D01E302D0006A02D0010E006E1200E6
:0A0ACC006B826BA201D0FDD712006F
:040AD6006B8412001B
:100ADA00A49E66C76FFF6DA401D0FDD7A4BE01D046
:100AEA00FDD76BBC02D0006A03D06B84020E006E85
:020AFA001200E8
:100AFC000701666B676B6751120802E166518E083D
:100B0C0009E332EC00F0005201E004D00701664B1F
:100B1C00672BF1D70701120E675D02E18F0E665D40
:100B2C0003E37B0E006E05D06B806BA001D0FDD76C
:040B3C00006A120039
:100B40005DC704F05EC705F05BC702F05CC703F049
:100B50005FC700F060C701F0010E07015F5F000E84
:100B6000605B005001100FE004C0E9FF05C0EAFF20
:100B700002C0E1FF03C0E2FFEECFE6FF024A032A14
:100B8000044A052AE5D75BC700F05CC701F01200F4
:100B90000B6A0C6A086A0350D8B44CEF06F002C026
:100BA0000AF0028E9E0E035E03AE3CEF06F0036C6D
:100BB000080E035CD8A009EF06F0036E083600C0EB
:100BC00008F001C000F002C001F0026A080E035CE8
:100BD000D8A009EF06F0036E083600C008F001C087
:100BE00000F0016A080E035CD8A009EF06F0036E5E
:100BF000083600C008F0006A080E035CD8A009EFB0
:100C000006F0036E0836086A0350D8A4D89015EF92
:100C100006F00350D8B415EF06F0D8900232013236
:100C200000320832032E0DEF06F00BBC08A026EFB1
:100C300006F0D8A026EF06F0082AD8B4002AD8B4C7
:100C4000012AD8B4022A02BE50EF06F00AAE4CEFD9
:100C500006F0021E011E001E081E082AD8B4002A33
:100C6000D8B4012AD8B4022A4CEF06F0026A016A0D
:100C7000006A086A4CEF06F00B800BAE56EF06F0E8
:100C8000026A0AAE56EF06F0026E016E006E086E42
:100C90000A36023256EF06F00C6A000E57EF06F0E5
:100CA000010E0C6E000E1FDE57EF06F0FF0E025015
:100CB000036E0150026E0050016E0850006E12006B
:100CC0005BC702F05CC703F002C000F003C001F094
:100CD000024A032A00C0E9FF01C0EAFFEE5201E028
:100CE000F3D707015B51025C006E5C510358016E43
:0A0CF000010E005E000E015A120012
:100CFA0007015E6B030E5E5D0AE25E515C25E16EE2
:100D0A00000E5D21E26E200EE66E5E2BF3D75E5179
:100D1A005C25E16E000E5D21E26EE66A5E075E51B9
:100D2A005C255F6F000E5D21606F0A0E046E5BC763
:100D3A0000F05DDE08C000F0300E00265FC7E1FF5C
:100D4A0060C7E2FF00C0E6FF0A0E046E5BC700F050
:100D5A004EDE00C05BF70050000A01E102D05E07D8
:040D6A00DED71200BE
:100D6E0007015D515E1108E05DC7E1FF5EC7E2FF5E
:100D7E005BC7E6FF5CC7E6FF5BC7E9FF5CC7EAFF40
:100D8E00EECF00F000C061F700C066F788DE0052BB
:100D9E0003E05B4B5C2BF0D75F6B000E61BFFF0E69
:100DAE00006E000E001802E12D0E611905E1010E14
:100DBE005F6F5B4B5C2B0CD0000E61BFFF0E006EA5
:100DCE00000E001802E12B0E611902E15B4B5C2B49
:100DDE00616B626B636B646B656B606B5FB90BD041
:100DEE005BC7E9FF5CC7EAFFEE502E0A04E15F899C
:100DFE005B4B5C2B52D05BC7E9FF5CC7EAFFEECFC3
:100E0E0066F7BBDD005201E149D05F836151080AEC
:100E1E003FE05FA901D06007612B62C700F063C796
:100E2E0001F064C702F065C703F00A0E046E000EEF
:100E3E00056E066E076E0ADE00C062F701C063F72C
:100E4E0002C064F703C065F7000000005BC7E9FF4E
:100E5E005CC7EAFF300EEE5C006E016A000E015AAE
:100E6E00000E01BEFF0E026E036E6251002663512C
:100E7E000122645102226551032200C062F701C0B3
:100E8E0063F702C064F703C065F70000000003D0EB
:100E9E005FB901D0602B5B4B5C2BA0D7616B5BC73E
:100EAE00E9FF5CC7EAFFEE50650A08E05BC7E9FFA1
:100EBE005CC7EAFFEE50450A01E065D05B4B5C2B48
:100ECE005BC7E9FF5CC7EAFFEE502D0A04E15F87BE
:100EDE005B4B5C2B09D05BC7E9FF5CC7EAFFEE50AA
:100EEE002B0A02E15B4B5C2B5BC7E9FF5CC7EAFF99
:100EFE00EE50300A03E15B4B5C2BF6D75BC7E9FF84
:100F0E005CC7EAFFEECF66F738DD005237E05BC70D
:100F1E00E9FF5CC7EAFF300EEE5C616F5B4B5C2B4A
:100F2E005BC7E9FF5CC7EAFFEECF66F726DD00522E
:100F3E0025E00A0E6103F3CF61F75BC7E9FF5CC7DB
:100F4E00EAFF300EEE5C006E005061275B4B5C2BAF
:100F5E005BC7E9FF5CC7EAFFEECF66F70EDD005216
:100F6E000DE00A0E6103F3CF61F75BC7E9FF5CC7C3
:100F7E00EAFF300EEE5C006E005061275FA703D0D3
:100F8E0061510008616F61516027000E5E1902E128
:100F9E00000E5D190AE05FA308D05DC7E1FF5EC7D2
:100FAE00E2FF5BC7E6FF5CC7E6FF62C700F063C700
:100FBE0001F064C702F065C703F026DD00C062F7DA
:100FCE0001C063F702C064F703C065F7046A056ADF
:100FDE00066A076A62C700F063C701F064C702F0D1
:100FEE0065C703F08BDC010ED8A4000E006E005214
:100FFE0005E0006A016A026A036A04D1800E601974
:10100E00006E800E000A005CD8B073D060510008EC
:10101E00606F800E6019006E800E0A0A005C1DE380
:10102E0062C700F063C701F064C702F065C703F042
:10103E00FF0E046EE60E056E5B0E066E5D0E076EFF
:10104E0097EC01F000C062F701C063F702C064F7CD
:10105E0003C065F70A0E605FDCD76051000A1CE022
:10106E0062C700F063C701F064C702F065C703F002
:10107E00CD0E046ECC0E056E4C0E066E7B0E076EFC
:10108E0097EC01F000C062F701C063F702C064F78D
:10109E0003C065F76007E1D7010E046E000E056E02
:1010AE00000E066E010E076E62C700F063C701F0F8
:1010BE0064C702F065C703F030EC01F0010ED8B042
:1010CE00000E006E005214E05FA109D0010E006EFA
:1010DE00000E016E800E026E030E036E93D0010E93
:1010EE00006E000E016E000E026E010E036E8AD0AF
:1010FE0072D0800E000A006E800E6019005C6BE2EA
:10110E000A0E605D1DE362C700F063C701F064C79D
:10111E0002F065C703F0F90E046E020E056E150E91
:10112E00066EA00E076E97EC01F000C062F701C0CC
:10113E0063F702C064F703C065F70A0E605FE0D77D
:10114E006051000A1CE062C700F063C701F064C77B
:10115E0002F065C703F0000E046E000E056E200E41
:10116E00066E820E076E97EC01F000C062F701C0AA
:10117E0063F702C064F703C065F76007E1D762C783
:10118E0004F063C705F064C706F065C707F0FF0EED
:10119E00006EFF0E016E7F0E026EFF0E036E30ECC0
:1011AE0001F0010ED8B0000E006E005214E05FA1E7
:1011BE0009D0FF0E006EFF0E016EFF0E026EFF0EC7
:1011CE00036E20D0FF0E006EFF0E016E7F0E026EBC
:1011DE00FF0E036E17D05FA10DD0000E6219006EC8
:1011EE00000E6319016E800E6419026E000E6519F1
:1011FE00036E08D062C700F063C701F064C702F047
:06120E0065C703F01200A9
:101214000450000A08E10550000A05E1FF0E006EC3
:101224007F0E016E58D00D6A096A086A01500010D9
:10123400D8B4000C015005180A6E0ABE0D1E0B6AC4
:1012440005AE05D0041E051E042AD8B4052A01AE35
:1012540005D0001E011E002AD8B4012A0150051031
:101264000A6E0ABE10D0D0EC04F00BB020D00DAE44
:10127400000C001E011E002AD8B4012A081E091EF3
:10128400082AD8B4092A000C05AE0DD001BE07D037
:101294000150096E0050086E016A006AE8D7016ABD
:1012A400006A002A000C011E001E0B2ADDD7082A42
:1012B400D8B4092A0450085CD8A4D9D70550095CCD
:1012C400D8A4D5D7096A086A002AD8B4012A01AE7D
:0812D400CED70000FF0C120050
:1012DC005BC7E9FF5CC7EAFFEECF5DF7000E0701C5
:1012EC005E6F000E5E6F000E5E1902E1200E5D193E
:1012FC0007E0000E5E1902E1090E5D1901E003D052
:10130C005B4B5C2BE5D75F6B606B616B626B000EAC
:10131C005E1902E12D0E5D1905E1614B622B5B4BF1
:10132C005C2B08D0000E5E1902E12B0E5D1902E158
:10133C005B4B5C2B5BC7E9FF5CC7EAFFEECF5DF74D
:10134C00000E5E6F000E5E6F5DC766F7C4EC04F0B6
:10135C00005219E05FC700F060C701F00A0E046E7E
:10136C00000E056E9CEC04F0300E5D5D026E000EFE
:10137C005E59036E025000245F6F03500120606FB2
:10138C005B4B5C2BD7D76151621108E05F510008B1
:10139C00006E60C701F0000E015604D05FC700F06C
:0613AC0060C701F0120011
:1013B200086A096A100E0C6E0134083609360450A8
:1013C200085E0550D8A0053C095ED8B007D004508D
:1013D20008260550D8B0053C0926D89000360136BB
:0613E2000C2EEAD71200F8
:1013E80000C008F00150006E016A026A036A0B6AC5
:1013F8000C6A016A026A036A960E036E0A6A00AEF4
:101408000CEF0AF0081E001E082AD8B4002A0A8E1B
:1014180000C001F008C000F0086A026A27EC02F078
:021428001200B0
:10142A000B6A0350D8B45BEF0AF002500A6E028EC0
:10143A008E0E035E03AE5FEF0AF0036C080E035CC8
:10144A00D8A03AEF0AF0036E013602C001F0026A30
:10145A00080E035CD8A03AEF0AF0036E0136016A5F
:10146A000350D8A4D89044EF0AF00350D8B444EFFC
:10147A000AF0D89002320132032E3EEF0AF00BBC7A
:10148A0001A051EF0AF0D8A051EF0AF0012AD8B40E
:10149A00022A02BE6EEF0AF00AAE74EF0AF0021ECA
:1014AA00011E012AD8B4022A74EF0AF0026A016AFC
:1014BA0074EF0AF00B800BAE78EF0AF0026A0AAEFC
:1014CA0078EF0AF0FF0E026E016E0A36023278EFEA
:1014DA000AF0010E0C6E73EC04F07AEF0AF0000EBB
:1014EA000C6E7AEF0AF0FF0E0C6E0150006E02507D
:0414FA00016E12006D
:1014FE005DC7F6FF5EC7F7FF5FC7F8FF0900F5CFC0
:10150E0000F0005218E05DC7F6FF5EC7F7FF5FC739
:10151E00F8FF0900F5CF00F05BC7E1FF5CC7E2FF03
:10152E0000C0E6FF07015B4B5C2B010E5D27000E32
:10153E005E235F23DDD75BC7E1FF5CC7E2FFE66A90
:02154E00120089
:0E155000A8B202D00000FCD75BC7A9FF1200B2
:10155E000450000A12E10550000A0FE10650000A7D
:10156E000CE10750000A09E1FF0E006EFF0E016E3E
:10157E007F0E026EFF0E036EA8D0086A096A07502E
:10158E00D8B45AEF0BF00350D8B45FEF0BF0025003
:10159E0006180A6E028E068E0E6A02C008F001C090
:1015AE000CF000C00DF004500D5E0550D8A0053CA7
:1015BE000C5E0650D8A0063C085E086A0C6A0D6ADE
:1015CE00D8A0F1EF0AF0D890023201320032083280
:1015DE00010E0E6E0750035ED8A0FEEF0AF07E0ECF
:1015EE000E240326D8B064EF0BF004EF0BF07E0E42
:1015FE000E240326D8A069EF0BF0180E0B6E0D36D5
:10160E000C3608360036013602360E360450005EB1
:10161E000550D8A0053C015E0650D8A0063C025EDF
:10162E0006340E120EA01FEF0BF00D802AEF0BF0FA
:10163E00045000260550D8B0053C01260650D8B0FF
:10164E00062802260D900B2E06EF0BF050EF0BF036
:10165E00D8900036013602360E360450005E055024
:10166E00D8A0053C015E0650D8A0063C025E0634AA
:10167E000E10010B0D26D8B00C2AD8B4082AD8A407
:10168E0050EF0BF008320C320D32032AD8B464EF4F
:10169E000BF00AAE089E0850026E0C50016E0D50F3
:1016AE00006E6CEF0BF0010E81EC04F06CEF0BF0A2
:1016BE00020E1AEC00F06CEF0BF0040E0EEC00F0C4
:0C16CE006CEF0BF0080E21EC00F0120095
:0E16DA00ADB202D00000FCD75BC7AEFF12001D
:1016E8007EEC05F08BC166F76DEC05F00701666BC3
:1016F8006DEC05F0020E0701666F6DEC05F00DD07C
:10170800800E0701666F6DEC05F015D0C00E07015D
:10171800666F6DEC05F00FD00ED0000E07015C1956
:1017280002E1010E5B19ECE0000E5C1902E1020E09
:101738005B19ECE0F1D766EC05F08BC166F76DEC50
:1017480005F0400E0701666F6DEC05F007015D6B53
:101758005E6B800E5E19006E800E005C04E1010174
:10176800895107015D5D08E2A00E666F6DEC05F01A
:1017780007015D4B5E2BEDD766EC05F08BC166F774
:101788006DEC05F00701666B6DEC05F00DD0800E71
:101798000701666F6DEC05F015D0C00E0701666F86
:1017A8006DEC05F00FD00ED0000E07015C1902E1B8
:1017B800010E5B19ECE0000E5C1902E1020E5B19E8
:0A17C800ECE0F1D76BEC05F0120025
:0817D200067E60EC02F012003B
:1017DA003DC704F03EC705F004C0E9FF05C0EAFFB3
:1017EA00EE5203E0044A052AF7D704C002F005C006
:1017FA0003F0044A052A3FC700F040C701F0070179
:10180A003F4B402B00C0E9FF01C0EAFF02C0E1FFE5
:10181A0003C0E2FFEECFE6FF02C0E9FF03C0EAFF22
:10182A00EE5201E0E2D73DC700F03EC701F01200D8
:10183A007EEC05F08BC166F76DEC05F00701666B6F
:10184A006DEC05F0000E006E07014051005C03E1EB
:10185A003F510101895D05E289C13FF7000E070189
:10186A00406F11D007013F51800F666F66076DEC1C
:10187A0005F017D007013F51C00F666F66076DEC80
:10188A0005F00FD00ED0000E07013E1902E1010E3D
:10189A003D19E8E0000E3E1902E1020E3D19EAE0A8
:1018AA00F1D766EC05F08BC166F76DEC05F0400EDA
:1018BA000701666F6DEC05F03FC743F740C744F771
:1018CA0041C7E9FF42C7EAFFEE521BE041C7D9FF11
:1018DA0042C7DAFFDE50800F0701666F6DEC05F034
:1018EA000701414B422B434B442B800E006E800E66
:1018FA004419005C03E143510101895D01E201D011
:08190A00DFD76BEC05F01200C1
:101912003DC7F6FF3EC7F7FF3FC7F8FF0900F5CF07
:1019220000F0005211E03DC7F6FF3EC7F7FF3FC788
:10193200F8FF0900F5CF5BF70ADE010E07013D272C
:0A194200000E3E233F23E4D71200FD
:10194C000701406B3DC7E9FF3EC7EAFFEECF3FF70B
:10195C003F51000A0EE03FC75BF7B9DE0701402B91
:10196C0040513D25E96E000E3E21EA6EEECF3FF769
:04197C00EFD712008F
:10198000530E07015B6F000E5C6FF70E5D6F560E16
:101990005E6F000E5F6FB3DD450E07015B6F070ED4
:1019A0005C6F3DC75DF73EC75EF7020E5F6F000ECE
:1019B000606FA0EC05F0D00E5024036E070E51208E
:1019C000046E03C000F004C001F001320032019E39
:1019D00001BC018E01320032019E01BC018E035018
:1019E000002604500122070E046E000E056E12DC64
:1019F00008C000F009C001F000C049F701C04AF773
:101A0000050E07014925006E000E4A21016E070EE2
:101A1000046E000E056E0AEC09F008C000F009C063
:101A200001F000501F0807014B6F01C04CF7000E7A
:101A30004C57020E4925006E000E4A21016E070E1A
:101A4000046E000E056E0AEC09F008C000F009C033
:101A500001F000501F080701496F01C04AF7000E4E
:101A60004A574EC000F04FC001F0640E046E000EE5
:101A7000056E9CEC04F000017B510024036E7C5148
:101A80000120046E03C041F704C042F72C0E070189
:101A90004B25016E010E4C21026EE80E4925436F65
:101AA000030E4A21446F306B316B800E0418006EB8
:101AB000800E0218005C02E10150035C1AE3800E04
:101AC0004419006E800E4219005C02E14151435DF1
:101AD00010E301018A8F450E07015B6F070E5C6FF3
:101AE0006EEC09F0020E00243F6F000E0120406FE3
:101AF0000FD001018A9F450E07015B6F070E5C6FD7
:101B00006EEC09F0010E00243F6F000E0120406FC3
:101B1000800E006E800E4019005C02E13F511708F4
:101B200006E23F6B406B010E306F000E316F3DC718
:101B30005BF73EC75CF760EC06F000C09FF001C0A9
:101B4000A0F03FC75BF7450E5C6F070E5D6F7DEC45
:101B500006F0530E5B6F000E5C6F460E5D6F070E56
:101B60005E6F020E5F6F000E606FA0EC05F0560E08
:101B70005B6F000E5C6F020E3D255D6F000E3E2117
:101B80005E6F020E5F6F000E606FA0EC05F0590EE5
:101B90005B6F000E5C6F040E3D255D6F000E3E21F5
:101BA0005E6F020E5F6F000E606FA0EC05F05E6A64
:021BB000120021
:101BB200400E07015B6F070E5C6F3DC75DF73EC7C6
:101BC2005EF73FC75FF79ADC7EEC05F08BC166F7E4
:101BD2006DEC05F00701666B6DEC05F066EC05F047
:101BE2008BC166F76DEC05F0400E0701666F6DEC78
:101BF20005F03DC7F6FF3EC7F7FF3FC7F8FF0900F4
:101C0200F5CF00F0005216E03DC7F6FF3EC7F7FFE2
:101C12003FC7F8FF0900F5CF00F00050800F070121
:101C2200666F6DEC05F0010E07013D27000E3E23A5
:0A1C32003F23DFD76BEC05F0120032
:101C3C00A49E6B86A4BE01D0FDD76FCF01F0070127
:101C4C003D51000A02E16B8A01D06B9AA49E6B880D
:0C1C5C00A4BE01D0FDD701C000F01200B2
:101C68003DC7F6FF3EC7F7FF3FC7F8FF0900F5CFAE
:101C780000F0005211E03DC7F6FF3EC7F7FF3FC72F
:101C8800F8FF0900F5CF5BF724DD010E07013D27BA
:0A1C9800000E3E233F23E4D71200A4
:101CA2003DC75BF73EC75CF707015D6B5E6BB7EC48
:041CB20006F0120026
:101CB60007014351000805E3070E446F000E456F08
:101CC60012D04351160805E2170E466F000E476FF5
:101CD60006D04351010F466F476B000E472346C798
:101CE60044F747C745F744C74EF745C74FF7486B14
:101CF600496B046A056A066A076A3DC700F03EC773
:101D060001F03FC702F040C703F030EC01F0010ECE
:101D1600D8B0000E006E005209E041C7E1FF42C78D
:101D2600E2FF2D0EE66E414B422B3F7F3DC704F08E
:101D36003EC705F03FC706F040C707F0006A016AD4
:101D4600026A036A30EC01F0010ED8B0000E006E94
:101D5600005237E0000E046E000E056E000E066E91
:101D66007F0E076E3DC700F03EC701F03FC702F089
:101D760040C703F030EC01F0010ED8B0000E006E43
:101D860000521FE03DC700F03EC701F03FC702F01A
:101D960040C703F0000E046E000E056E200E066EA0
:101DA600820E076E97EC01F000C03DF701C03EF7CA
:101DB60002C03FF703C040F7010E485F000E495BC3
:101DC600C9D7000E046E000E056E200E066E820E3A
:101DD600076E3DC700F03EC701F03FC702F040C79F
:101DE60003F030EC01F0000ED8B0010E006E005288
:101DF6001EE0000E046E000E056E200E066E820EAC
:101E0600076E3DC700F03EC701F03FC702F040C76E
:101E160003F0AFEC0AF000C03DF701C03EF702C088
:101E26003FF703C040F70701484B492BCAD7485133
:101E36004E2749514F23010E4A6F000E4B6F000E7D
:101E4600506F000E516F000E526F7F0E536F800E53
:101E56004B19006E800E4F19005C02E14E514A5D2F
:101E66001EE2000E046E000E056E200E066E820E39
:101E7600076E50C700F051C701F052C702F053C7B2
:101E860003F0AFEC0AF000C050F701C051F702C0F2
:101E960052F703C053F707014A4B4B2BD8D7000E16
:101EA600046E000E056E000E066E800E076E50C79D
:101EB60000F051C701F052C702F053C703F0AFEC70
:101EC6000AF03DC704F03EC705F03FC706F040C71D
:101ED60007F060EC02F000C03DF701C03EF702C01B
:101EE6003FF703C040F7000E046E000E056E200E8D
:101EF600066E820E076E30EC01F0000ED8B0010EB1
:101F0600006E00520BE0000E07013D6F000E3E6FA3
:101F1600000E3F6F7F0E406F484B492B0701800E26
:101F26004919006E800E005C02E1000E485D38E241
:101F360041C7E1FF42C7E2FF300EE66E414B422B3E
:101F460041C7E1FF42C7E2FF2E0EE66E414B422B30
:101F5600800E4F19006E800E005C02E1000E4E5D91
:101F660004E24E51485F4F51495BFF0E4A6FFF0E28
:101F76004B6F800E4919006E800E4B19005C02E112
:101F86004A51485D0DE241C7E1FF42C7E2FF300E0C
:101F9600E66E414B422B010E4A5F000E4B5BE9D7C2
:101FA6004A6B4B6B800E4B19006E800E4F19005C0E
:101FB60002E14E514A5D63E23DC700F03EC701F0C3
:101FC6003FC702F040C703F015EC0AF000C04CF71B
:101FD60001C04DF7300E002641C7E1FF42C7E2FFC0
:101FE60000C0E6FF414B422B4B51491902E14851D3
:101FF6004A1908E141C7E1FF42C7E2FF2E0EE66E2D
:10200600414B422B4CC700F04DC701F0F4EC09F0F0
:1020160000C050F701C051F702C052F703C053F792
:1020260000C004F001C005F002C006F003C007F0CE
:102036003DC700F03EC701F03FC702F040C703F0BE
:10204600E9EC0BF000C03DF701C03EF702C03FF7D8
:1020560003C040F7000E046E000E056E200E066EDD
:10206600820E076E97EC01F000C03DF701C03EF707
:1020760002C03FF703C040F74A4B4B2B93D741C7EB
:0A208600E1FF42C7E2FFE66A120024
:102090000D0E07015B6F6DEC0BF00A0E07015B6F15
:0620A0006DEC0BF01200D4
:1020A600440E07015B6F070E5C6F41C75DF742C7C1
:1020B6005EF743C75FF77FEC0AF07EEC05F08BC155
:1020C60066F76DEC05F00701666B6DEC05F0000E2A
:1020D600006E07014051005C03E13F510101895D3B
:1020E60005E289C13FF7000E0701406F11D00701D5
:1020F6003F51800F666F66076DEC05F017D007013C
:102106003F51C00F666F66076DEC05F00FD00ED01D
:10211600000E07013E1902E1010E3D19E8E0000E2E
:102126003E1902E1020E3D19EAE0F1D766EC05F030
:102136008BC166F76DEC05F0400E0701666F6DEC1E
:1021460005F03FC759F740C75AF741C7F6FF42C7E0
:10215600F7FF43C7F8FF0900F5CF00F0005223E070
:1021660041C7F6FF42C7F7FF43C7F8FF0900F5CF9F
:1021760000F00050800F0701666F6DEC05F0010E50
:1021860007014127000E42234323594B5A2B800E49
:10219600006E800E5A19005C03E159510101895DF8
:0C21A60001E201D0D2D76BEC05F0120072
:1021B20007013F6B406B3DC703F03EC704F03DC7CC
:1021C20005F03EC706F003C0E9FF04C0EAFFEE5087
:1021D200200A04E13F51401101E110D0010E3F6F8E
:1021E200000E406F03C0E9FF04C0EAFF05C0E1FF33
:1021F20006C0E2FFEECFE6FF054A062A03C001F061
:1022020004C002F0034A042A01C0E9FF02C0EAFF47
:10221200EE50000AD8E13DC700F03EC701F01200BF
:1022220041C700F007014107005228E03DC7E9FF1E
:102232003EC7EAFFEE50000A0CE03DC7E9FF3EC789
:10224200EAFF3FC7D9FF40C7DAFFEE50DE1801E1CF
:102252000FD03DC7E9FF3EC7EAFF3FC7D9FF40C7DE
:10226200DAFFDE50EE5C006E016A000E015A08D001
:1022720007013D4B3E2B3F4B402BD2D7006A016AF0
:02228200120048
:1022840040C700F0016A026A036AFF0E0016000EDE
:10229400011600C045F701C046F77F0E005C026ED0
:1022A400000E0158036E02C045F703C046F7800EC6
:1022B4000318006E800E005C02E1000E025C22E254
:1022C400046A056A066A076A3DC700F03EC701F062
:1022D4003FC702F040C703F030EC01F0010ED8B064
:1022E400000E006E005209E0000E006E000E016E3A
:1022F400800E026E7F0E036E5ED0006A016A026A6F
:10230400036A59D0000E006E07014651005C02E1D9
:102314004551180809E23DC700F03EC701F03FC728
:1023240002F040C703F047D03DC700F03EC701F0BC
:102334003FC702F040C703F0C8EC05F00BEC05F012
:1023440000C041F701C042F702C043F703C044F79D
:1023540000C004F001C005F002C006F003C007F09D
:102364003DC700F03EC701F03FC702F040C703F08D
:1023740030EC01F0010ED8B0000E006E005213E0F4
:10238400000E046E000E056E000E066E7F0E076EC4
:1023940041C700F042C701F043C702F044C703F04D
:1023A400E9EC0BF008D041C700F042C701F043C785
:0823B40002F044C703F012001F
:1023BC000701416B050E415D0AE241513F25E16E7B
:1023CC00000E4021E26E200EE66E412BF3D74151F8
:1023DC003F25E16E000E4021E26EE66A4107415155
:1023EC003F25426F000E4021436F0A0E046E000E13
:1023FC00056E3DC700F03EC701F0D9EC09F008C0EE
:10240C0000F009C001F0300E002642C7E1FF43C7BF
:10241C00E2FF00C0E6FF0A0E046E000E056E3DC71B
:10242C0000F03EC701F0D9EC09F000C03DF701C047
:10243C003EF7000E011802E1000E001801E102D077
:06244C004107CDD712008C
:10245200020E07015B6F000E5C6F74EC0BF0010E55
:0E24620007015B6F000E5C6F74EC0BF0120054
:102470003DC7E9FF3EC7EAFFEE5007013F1905E1FE
:102480003DC700F03EC701F010D03DC700F03EC789
:1024900001F03D4B3E2B00C0E9FF01C0EAFFEECF4B
:0C24A00000F00052E5E1006A016A120041
:1024AC003DC704F03EC705F004C002F005C003F0C0
:1024BC00044A052A3FC700F040C701F007013F4B13
:1024CC00402B00C0E9FF01C0EAFF02C0E1FF03C0DE
:1024DC00E2FFEECFE6FF02C0E9FF03C0EAFFEE52D7
:0E24EC0001E0E2D73DC700F03EC701F012004C
:1024FA00500E07012C6F150E2D6F5B0E2E6F070EF7
:10250A002F6FFF0E286FFF0E296F000E2A6F000E25
:10251A002B6FFF0E0401A56FFF0EA66F000EA76FAB
:10252A00000EA86FFF0EA16FFF0EA26F000EA36F21
:10253A00000EA46FA88A900E9C6E98849892A4AA02
:0A254A0003D0AACF00F0FBD7120067
:102554000900F5CFE6FF0006FBE10106F9E11200F0
:10256400959A959C8C9A8C9C958A958C6D9E6D9C65
:06257400380E6C6E12002F
:10257A000401AF6BB06B020EB05D02E1000EAF5DFD
:10258A000AE2B60EAF25E16E040EB021E26EE66AEB
:10259A00AF4BB02BF0D7AD6BAE6BAF6BB06B9EAAE7
:1025AA0002D0AFCFB5F4B56B9F6BA06BA08A1200B7
:1025BA00DA0E07012C6F160E2D6F5B0E2E6F070EAB
:1025CA002F6FFF0E286FFF0E296F000E2A6F000E65
:1025DA002B6FFF0E0401A56FFF0EA66F000EA76FEB
:1025EA00000EA86FFF0EA16FFF0EA26F000EA36F61
:1025FA00000EA46FAD8A900EAC6E948E949C9EAA27
:0A260A0003D0AFCF00F0FBD71200A1
:10261400FF0E926EFD0EC16EFF0EC26E9384FF0E0E
:10262400936EFF0E956EFF0E946EFF0E986E959C42
:10263400958E9986959896988C988D989380938288
:02264400120082
:10264600E90E07013D6F550E3E6F000E3F6F34ECED
:102656000EF032C75BF7340E07015C6F070E5D6F35
:102666007DEC06F0340E3D6F070E3E6FA6EC0CF0C7
:10267600A00E3D6F570E3E6F000E3F6F34EC0EF00E
:10268600670E07013D6F570E3E6F000E3F6F34EC2D
:102696000EF07EEC05F032C766F76DEC05F000C073
:1026A60033F70050000A0CE0A80E07013D6F560EE6
:1026B6003E6F000E3F6F34EC0EF00701336B0CD00B
:1026C60007012E0E3D6F570E3E6F000E3F6F34EC26
:1026D6000EF0010E0701336F6BEC05F0D6DC33C745
:0426E60000F01200EE
:1026EA000701346B356B1F0E0B6E710E0C6E1E0ECE
:1026FA000D6E0D2EFED70C2EFCD70B2EFAD700002E
:10270A007EEC05F08BC166F76DEC05F000C032F780
:10271A00000E0701336F000E331902E1000E321961
:10272A0005E034C700F035C701F0C9D0344B352B6A
:10273A000D0E0B6E2D0E0C6ED70E0D6E0D2EFED7D6
:10274A000C2EFCD70B2EFAD700000000666B6DEC3E
:10275A0005F000C032F7000E0701336F800E006EDD
:10276A00800E3319005C02E13251000805E234C7D9
:10277A0000F035C701F0A3D0344B352B240E666F19
:10278A006DEC05F00C0E0701666F6DEC05F0060E98
:10279A000701666F6DEC05F0250E0701666F6DEC9B
:1027AA0005F0060E0701666F6DEC05F0110E0701C4
:1027BA00666F6DEC05F0420E0701666F6DEC05F071
:1027CA00960E0701666F6DEC05F0240E0701666F21
:1027DA006DEC05F000C032F7000E0701336F800E72
:1027EA00006E800E3319005C02E13251000805E2E6
:1027FA0034C700F035C701F062D0344B352B0C0ECC
:10280A00666F6DEC05F000C032F7000E0701336FFA
:10281A00800E006E800E3319005C02E1325100080E
:10282A0005E234C700F035C701F049D0344B352BE7
:10283A00060E666F6DEC05F000C032F7000E070158
:10284A00336F800E006E800E3319005C02E1325144
:10285A00000805E234C700F035C701F030D0344B28
:10286A00352B020E666F6DEC05F000C032F7000ED4
:10287A000701336F800E006E800E3319005C02E18F
:10288A003251000805E234C700F035C701F017D00D
:10289A00344B352B070E0B6E170E0C6E6A0E0D6E2F
:1028AA000D2EFED70C2EFCD70B2EFAD700006BECA0
:1028BA0005F0344B352B34C700F035C701F0120050
:1028CA00150E7B6EA00E7A6E0601BA6BBB6B7992FF
:1028DA00798A7988799C79967994798E7990A29275
:0628EA00A192A092120071
:1028F000FF0E0401B16FFF0EB26FFF0EB36FFF0E3C
:0E290000B46FC26A070EC16EC18EC280120093
:10290E000701356B32C7E9FF33C7EAFFEECF34F765
:10291E003451000A0FE034C75BF7A8EC0AF0070148
:10292E00352B35513225E96E000E3321EA6EEECF8E
:06293E0034F7EED7120091
:102944000D0E07015B6FA8EC0AF00A0E07015B6F1E
:06295400A8EC0AF01200DD
:10295A000401996B9A6BF2AE03D0010E0701366F30
:10296A00F29E090E006E32C703F033C704F000501E
:10297A0005E004320332049EFF0FFAD703C000F0C9
:10298A0004C001F000360090013600C034F701C0DF
:10299A0035F70050A00F0401986F070E006E32C77A
:1029AA0034F733C735F7005006E00701343734915E
:1029BA003537FF0FF9D77EEC05F098C466F76DEC52
:1029CA0005F035C766F76DEC05F034C766F76DECB0
:1029DA0005F00050000803E20401994B9A2B070105
:1029EA00346B356B000E355D02E17F0E345D1CE2FF
:1029FA00160E3425E96E040E3521EA6EEECF66F71F
:102A0A006DEC05F00050000803E20401994B9A2B83
:102A1A004E0E0C6EEB0E0D6E0D2EFED70C2EFCD745
:102A2A000701344B352BDED76BEC05F032EC00F0A6
:0C2A3A0007013651010AD8B4F28E1200D8
:102A4600010E07015B6F000E5C6F74EC0BF00E0E4F
:102A560007015B6F010E5C6FB60E5D6F550E5E6F04
:102A6600000E5F6F7FEC0AF0860E07015B6F000EAB
:102A76005C6F60EC06F000500608026E01C003F0C1
:102A8600000E035602C032F703C033F7800E031858
:102A9600006E800E005C02E1000E025C02E2326B08
:102AA600336B325119083D6F33C73EF7010E3E575F
:102AB600860E3F6F000E406FF6DC6D0E01011D6F36
:102AC600010E07013D6F000E3E6F010E3F6F000EB7
:102AD600406F0E0E416F010E426F1DEC0CF0020EA0
:102AE60007015B6F000E5C6F74EC0BF0BC0E070108
:102AF6003D6F060E3E6FC0EC0CF0020E3D6F000EF1
:102B06003E6F010E3F6F000E406FB70E416F570EBE
:102B1600426F000E436F53EC10F0020E07013D6F3B
:102B2600000E3E6F070E3F6F000E406F530E416F53
:102B3600000E426F1DEC0CF05C0E0B6E510E0C6E0F
:102B4600600E0D6E0D2EFED70C2EFCD70B2EFAD76F
:102B560000000E0E07015B6F010E5C6FC70E5D6F06
:102B6600550E5E6F000E5F6F7FEC0AF09BC43DF75B
:102B76009CC43EF79DC43FF79EC440F7130E070161
:102B8600416F010E426F060E436F5BEC0EF00E0EA8
:102B96005B6F010E5C6F60EC06F0800E0118026E32
:102BA600800E025C02E1100E005C0BE20E0E3D6F21
:102BB600010E3E6F1D0E3F6F000E406FEDEC0BF0E9
:102BC600E6D79EC01DF101011E6B010E07013D6F88
:102BD600000E3E6F010E3F6F000E406F0E0E416FEE
:102BE600010E426F1DEC0CF00E0E07015B6F010E1D
:102BF6005C6FA50E5D6F550E5E6F000E5F6F7FEC0E
:102C06000AF04EC13DF74FC13EF750C13FF751C1E3
:102C160040F7130E0701416F010E426F060E436F18
:102C26005BEC0EF00E0E5B6F010E5C6F60EC06F057
:102C3600800E0118026E800E025C02E1100E005C2E
:102C46000BE20E0E3D6F010E3E6F1F0E3F6F000E24
:102C5600406FEDEC0BF0E6D70DC11DF101011E6BC7
:102C6600020E07013D6F000E3E6F010E3F6F000E14
:102C7600406F0E0E416F010E426F1DEC0CF05C0EA4
:102C86000B6E510E0C6E600E0D6E0D2EFED70C2EB9
:102C9600FCD70B2EFAD700005DC15BF75EC15CF76F
:102CA6001C0E07015D6F560E5E6F000E5F6F7FECA8
:102CB6000AF0080E01015D25E16E000E5E21E26E4E
:102CC60096C0E6FF090E5D25E16E000E5E21E26EFE
:102CD60097C0E6FF0F0E5D25E16E000E5E21E26EE7
:102CE6000CC1E6FF100E5D25E16E000E5E21E26E60
:102CF600E66A8BC18EF129EC12F0010E07013D6FD9
:102D0600000E3E6F010E3F6F000E406F5DC141F732
:102D16005EC142F71DEC0CF001010351000A21E1EE
:102D2600020E07013D6F000E3E6F010E3F6F000E53
:102D3600406FFA0E416F550E426F000E436F53EC13
:102D460010F0020E07013D6F000E3E6F070E3F6F3B
:102D5600000E406F7D0E416F000E426F1DEC0CF0B1
:102D660076D001010E6B5DC15BF75EC15CF7BE0EEE
:102D760007015D6F570E5E6F000E5F6F7FEC0AF006
:102D86008FC13DF790C13EF70E0E07013F6F010E52
:102D9600406FDEEC11F00E0E3D6F010E3E6FD9EC6A
:102DA60010F000C08CF101C08DF18CC15BF78DC1B4
:102DB6005CF760EC06F0800E0118026E800E025C75
:102DC60002E1050E005C0BE28CC13DF78DC13EF7BA
:102DD600210E3F6F000E406FEDEC0BF0E6D75DC1A4
:102DE6003DF75EC13EF78CC13FF78DC140F7EDEC74
:102DF6000BF05DC13DF75EC13EF7230E3F6F000E3F
:102E0600406FEDEC0BF00F0E01015D25E16E000E3B
:102E16005E21E26E04019651300F006E00C0E6FF9F
:102E2600100E01015D25E16E000E5E21E26EE66A7E
:102E3600020E07013D6F000E3E6F010E3F6F000E42
:102E4600406F5DC141F75EC142F71DEC0CF0120008
:102E5600000E0701331902E1000E321937E032C7BE
:102E6600E9FF33C7EAFFEE5231E034C75BF735C7F7
:102E76005CF760EC06F000C041F732C73DF733C798
:102E86003EF734C73FF735C740F711EC11F0000E97
:102E9600011802E1000E001805E132C700F033C741
:102EA60001F016D0010E070132253D6F000E3321C9
:102EB6003E6F34C7E9FF35C7EAFFEECF3FF738EC80
:102EC60012F000C032F701C033F7C2D7006A016AB8
:022ED6001200E8
:102ED80032C704F033C705F007013651371124E033
:102EE800010E365F000E375B04C002F005C003F028
:102EF800044A052A34C700F035C701F0344B352B96
:102F080000C0E9FF01C0EAFF02C0E1FF03C0E2FF21
:102F1800EECFE6FF02C0E9FF03C0EAFFEECF00F004
:102F2800005201E101D0D8D736C700F037C701F009
:102F3800010E365F000E375B0050011008E004C038
:102F4800E1FF05C0E2FFE66A044A052AEDD732C769
:082F580000F033C701F0120084
:102F60000401996B9A6BF2AE03D0010E0701366F24
:102F7000F29E090E006E32C703F033C704F0005012
:102F800005E004320332049EFF0FFAD703C000F0BD
:102F900004C001F000360090013600C034F701C0D3
:102FA00035F70050A00F0401986F070E006E32C76E
:102FB00034F733C735F7005006E007013437349152
:102FC0003537FF0FF9D77EEC05F098C466F76DEC46
:102FD00005F035C766F76DEC05F034C766F76DECA4
:102FE00005F00050000803E20401994B9A2B66ECAF
:102FF00005F004019851010F0701666F6DEC05F0B3
:1030000032EC00F00701346B356B000E355D02E1E8
:103010007E0E345D14E2160E3425376F040E352112
:10302000386F010E3D6F1EEC0EF037C7E1FF38C759
:10303000E2FF00C0E6FF0701344B352BE6D7160E42
:103040003425376F040E3521386F3D6B1EEC0EF0C2
:1030500037C7E1FF38C7E2FF00C0E6FF6BEC05F0C1
:1030600032EC00F0040E0B6E0C0E0C6E330E0D6E77
:103070000D2EFED70C2EFCD70B2EFAD70000000029
:0C30800007013651010AD8B4F28E12008C
:10308C00150E7B6EA00E7A6E0601BA6BBB6BA1920D
:06309C00A0827980120001
:1030A2000101016B026B020E025D02E1000E015D85
:1030B2000AE2140E0125E16E020E0221E26EE66AB8
:1030C200014B022BF0D70401146B156B0101016B4C
:1030D200026BA4AA02D0AACF13F20201136B010160
:0830E200916B926BA38A1200AE
:1030EA00010E07015B6F000E5C6F74EC0BF0440E6F
:1030FA0007013D6F550E3E6F000E3F6FD9EC0DF084
:10310A00020E07015B6F000E5C6F74EC0BF04E0E43
:10311A0007013D6F560E3E6F000E3F6FD9EC0DF062
:10312A00C70E07013D6F570E3E6F000E3F6F89ECC9
:10313A000CF01F0E0B6E710E0C6E1E0E0D6E0D2E08
:10314A00FED70C2EFCD70B2EFAD70000020E070171
:10315A005B6F000E5C6F74EC0BF05D0E07013D6F48
:10316A00560E3E6F000E3F6FD9EC0DF01F0E0B6E20
:10317A00710E0C6E1E0E0D6E0D2EFED70C2EFCD788
:10318A000B2EFAD70000230E07013D6F570E3E6F34
:10319A00000E3F6F89EC0CF01F0E0B6E710E0C6E59
:1031AA001E0E0D6E0D2EFED70C2EFCD70B2EFAD747
:1031BA000000020E07015B6F000E5C6F74EC0BF0EF
:1031CA00990E07013D6F560E3E6F000E3F6FD9EC08
:1031DA000DF01F0E0B6E710E0C6E1E0E0D6E0D2E67
:1031EA00FED70C2EFCD70B2EFAD70000930E070140
:1031FA003D6F550E3E6F000E3F6F89EC0CF03D0E91
:10320A000B6EE10E0C6E3F0E0D6E0D2EFED70C2EC0
:10321A00FCD70B2EFAD700000000020E07015B6FE5
:10322A00000E5C6F74EC0BF0010E07015B6F000E71
:10323A005C6F74EC0BF07B0E07013D6F560E3E6F10
:10324A00000E3F6FD9EC0DF01F0E0B6E710E0C6E57
:10325A001E0E0D6E0D2EFED70C2EFCD70B2EFAD796
:04326A00000012004E
:10326E00BC0E07013D6F060E3E6FC0EC0CF0530E08
:10327E003D6F000E3E6FA6EC0CF0A80E3D6F570E84
:10328E003E6F000E3F6F34EC0EF03A0E07013D6FAD
:10329E00010E3E6F51EC0EF000C09BF401C09CF489
:1032AE0002C09DF403C09EF4000E046E000E056E67
:1032BE00480E066E850E076EAFEC0AF000C04AF19E
:1032CE0001C04BF102C04CF103C04DF100C03DF7FF
:1032DE0001C03EF702C03FF703C040F742EC11F0C9
:1032EE0000C032F701C033F702C034F703C035F720
:1032FE0032C74AF133C74BF134C74CF135C74DF1E4
:10330E00000E046E000E056E480E066E850E076EDC
:10331E009BC400F09CC401F09DC402F09EC403F057
:10332E00AFEC0AF032C704F033C705F034C706F02D
:10333E0035C707F0E9EC0BF000C036F101C037F1EC
:10334E0002C038F103C039F1000E046E000E056E96
:10335E00480E066E850E076E97EC01F0000E046E99
:10336E00000E056E700E066E840E076EAFEC0AF040
:10337E0032C704F033C705F034C706F035C707F07F
:10338E0060EC02F000C09BF401C09CF402C09DF4FE
:10339E0003C09EF401010D51530A1AE19BC400F0C3
:1033AE009CC401F09DC402F09EC403F0000E046E96
:1033BE00000E056E800E066E7F0E076E97EC01F006
:1033CE0000C09BF401C09CF402C09DF403C09EF4A7
:1033DE009BC43DF79CC43EF79DC43FF79EC440F787
:1033EE000E0E0701416F010E426F060E436F5BEC2E
:1033FE000EF00E0E3D6F010E3E6FA6EC0CF00101AD
:10340E005F6B606B000E605D02E1280E5F5D0BE28C
:10341E00610E5F25E16E010E6021E26E200EE66EFA
:10342E005F4B602BEFD7616B886B610E07013D6FB1
:10343E00010E3E6F0E0E3F6F010E406F56EC12F0F6
:10344E005DC15BF75EC15CF7CA0E5D6F570E5E6FB6
:10345E00000E5F6F7FEC0AF0610E07013D6F010EEB
:10346E003E6F5DC13FF75EC140F7EDEC0BF0200EF5
:10347E005B6F6DEC0BF00DC15BF76DEC0BF04C0E52
:10348E0007013D6F570E3E6F000E3F6F34EC0EF08E
:10349E00520E07013D6F010E3E6F51EC0EF000C053
:1034AE004EF101C04FF102C050F103C051F1000EB8
:1034BE00046E000E056E480E066E850E076EAFEC9E
:1034CE000AF000C04AF101C04BF102C04CF103C03A
:1034DE004DF100C03DF701C03EF702C03FF703C0FB
:1034EE0040F742EC11F000C032F701C033F702C0D2
:1034FE0034F703C035F732C74AF133C74BF134C73F
:10350E004CF135C74DF1000E046E000E056E480EDF
:10351E00066E850E076E4EC100F04FC101F050C110
:10352E0002F051C103F0AFEC0AF032C704F033C71A
:10353E0005F034C706F035C707F0E9EC0BF000C014
:10354E0036F101C037F102C038F103C039F1000E77
:10355E00046E000E056E480E066E850E076E97EC15
:10356E0001F0000E046E000E056E700E066E840ED7
:10357E00076EAFEC0AF032C704F033C705F034C75C
:10358E0006F035C707F060EC02F000C04EF101C046
:10359E004FF102C050F103C051F100019E51570A84
:1035AE001AE14EC100F04FC101F050C102F051C1FD
:1035BE0003F0000E046E000E056E800E066E7F0E7A
:1035CE00076E97EC01F000C04EF101C04FF102C042
:1035DE0050F103C051F14EC13DF74FC13EF750C1FE
:1035EE003FF751C140F70E0E0701416F010E426FBA
:1035FE00060E436F5BEC0EF00E0E3D6F010E3E6F2E
:10360E00A6EC0CF0200E5B6F6DEC0BF09EC05BF722
:10361E006DEC0BF0610E07013D6F010E3E6F0E0E4D
:10362E003F6F010E406FEDEC0BF0610E5B6F010E04
:10363E005C6F60EC06F000C09FF001C0A0F0610E60
:10364E000024E16E010E0120E26E2C0EE66E010EDC
:10365E0000019F25006E000EA021016E610E002458
:10366E00E16E010E0120E26EE66ADF0E07013D6F8C
:10367E00560E3E6F000E3F6F34EC0EF0860E0701B5
:10368E003D6F000E3E6F51EC0EF000C09AF001C07F
:10369E009BF002C09CF003C09DF000C03DF701C03E
:1036AE003EF702C03FF703C040F70E0E416F010E0A
:1036BE00426F010E436F5BEC0EF0610E3D6F010E1B
:1036CE003E6F0E0E3F6F010E406FEDEC0BF00E0EC7
:1036DE003D6F010E3E6FA6EC0CF0610E5B6F010E9E
:1036EE005C6F60EC06F000C09FF001C0A0F0610EB0
:1036FE000024E16E010E0120E26E2C0EE66E010E2C
:10370E0000019F25006E000EA021016E610E0024A7
:10371E00E16E010E0120E26E96C0E6FF020E9F25BD
:10372E00006E000EA021016E610E0024E16E010EEE
:10373E000120E26E97C0E6FF030E9F25006E000E7D
:10374E00A021016E610E0024E16E010E0120E26ED9
:10375E00E66A0101806B180E07013D6F570E3E6F32
:10376E00000E3F6F34EC0EF0960E07013D6F000E0B
:10377E003E6FA6EC0CF0EB0E3D6F560E3E6F000E3C
:10378E003F6F34EC0EF0040E07013D6F010E3E6FDD
:10379E00A6EC0CF0420E3D6F570E3E6F000E3F6FC3
:1037AE0034EC0EF00CC15BF76DEC0BF0020E070162
:1037BE003D6F570E3E6F000E3F6F34EC0EF0300E25
:1037CE000101032507015B6F6DEC0BF048EC10F067
:0237DE001200D7
:1037E0000701346B356B010E386F000E396FA10E77
:1037F0005B6F000E5C6F60EC06F000C036F701C036
:1038000037F7070E326F000E336F800E3319006EDC
:10381000800E3719005C02E13651325DD8B089D193
:1038200046D1A10E3225E96E000E3321EA6EEE502C
:103830002C0A0EE1BC0E3425E16E060E3521E26E37
:10384000E66A346B356B020E386F000E396F6ED13D
:10385000BC0E3425E16E060E3521E26EA10E322536
:10386000E96E000E3321EA6EEECFE6FF344B352BC6
:103870005DD1A10E3225E96E000E3321EA6EEE50C5
:103880002C0A0EE1520E3425E16E010E3521E26E56
:10389000E66A346B356B030E386F000E396F46D114
:1038A000520E3425E16E010E3521E26EA10E322555
:1038B000E96E000E3321EA6EEECFE6FF344B352B76
:1038C00035D1A10E3225E96E000E3321EA6EEE509D
:1038D0002C0A07E1346B356B040E386F000E396F1C
:1038E00025D1A10E3225E96E000E3321EA6EEECF0E
:1038F0000DF1344B352B1AD1A10E3225E96E000E95
:103900003321EA6EEE502C0A0EE13A0E3425E16EB8
:10391000010E3521E26EE66A346B356B050E386FA9
:10392000000E396F03D13A0E3425E16E010E3521B8
:10393000E26EA10E3225E96E000E3321EA6EEECF63
:10394000E6FF344B352BF2D0A10E3225E96E000E86
:103950003321EA6EEE502C0A07E1346B356B060E0C
:10396000386F000E396FE2D0A10E3225E96E000EDD
:103970003321EA6EEECF9EF0344B352BD7D0A10E1B
:103980003225E96E000E3321EA6EEE502C0A07E173
:10399000346B356B070E386F000E396FC7D0A10E30
:1039A0003225E96E000E3321EA6EEECF0CF1344B76
:1039B000352BBCD0A10E3225E96E000E3321EA6E04
:1039C000EE502C0A0EE1960E3425E16E000E3521E4
:1039D000E26EE66A346B356B080E386F000E396F95
:1039E000A5D0960E3425E16E000E3521E26EA10EB3
:1039F0003225E96E000E3321EA6EEECFE6FF344B3E
:103A0000352B94D0A10E3225E96E000E3321EA6EDB
:103A1000EE502C0A0EE1040E3425E16E010E352124
:103A2000E26EE66A346B356B090E386F000E396F43
:103A30007DD0040E3425E16E010E3521E26EA10E1B
:103A40003225E96E000E3321EA6EEECFE6FF344BED
:103A5000352B6CD0A10E3225E96E000E3321EA6EB3
:103A6000EE502C0A0EE1860E3425E16E000E352153
:103A7000E26EE66A346B356B0A0E386F000E396FF2
:103A800055D0860E3425E16E000E3521E26EA10E72
:103A90003225E96E000E3321EA6EEECFE6FF344B9D
:103AA000352B44D036C732F737C733F73FD0000E37
:103AB000391902E1010E3819D8B4B3D6000E3919FC
:103AC00002E1020E3819D8B4D4D6000E391902E139
:103AD000030E3819D8B4F5D6000E391902E1040ED8
:103AE0003819D8B409D7000E391902E1050E381972
:103AF000D8B42AD7000E391902E1060E3819D8B405
:103B00003ED7000E391902E1070E3819D8B452D742
:103B1000000E391902E1080E3819D8B473D7000E17
:103B2000391902E1090E381995E0BCD7324B332B15
:0C3B30006CD638C700F039C701F0120055
:103B3C007D0E07015B6F000E5C6F550E5D6F570EAF
:103B4C005E6F000E5F6F7FEC0AF0FDC67DF0FEC667
:103B5C007EF0FFC680F000C781F001C783F002C77A
:103B6C0084F00001856B7D0E07013D6F000E3E6FEA
:103B7C00A6EC0CF0200E5B6F6DEC0BF0200E070129
:103B8C005B6F6DEC0BF0300E0601FD5D006E016A93
:103B9C00000E015A0A0E046E000E056E9CEC04F029
:103BAC00FE51002400017B6F000E01207C6F300E53
:103BBC007B5F000E7C5B0701305100017B27070106
:103BCC00315100017C23300E0601FF5D006E016A4D
:103BDC00000E015A0A0E046E000E056E9CEC04F0E9
:103BEC000701005100244E6E000E01204F6E300E66
:103BFC004E5E000E4F5A300E015D006E016A000ED3
:103C0C00015A0A0E046E000E056E9CEC04F0025173
:103C1C000024506E000E0120516E300E505E000ECE
:043C2C00515A1200D7
:103C300000C01AF0E1CF1BF0E2CF1CF09EAA49D0E1
:103C40009DAA47D0ACA203D0AC98AC88AC92ACA4EF
:103C500002D0AFCFB5F4AFCFB5F40401B5510D0A22
:103C600007E0020EB05D02E1000EAF5D01E223D07D
:103C7000010E9F6F000EA06F020EB05D02E1000EFC
:103C8000AF5D04E3020E9F6F000EA06FA09AB60E08
:103C9000AF25E16E040EB021E26EE66AAFC4ADF46A
:103CA000B0C4AEF4AF6BB06B9EBA01D0FDD7AFCF4E
:103CB000B5F4B56B0ED0B60EAF25E16E040EB02193
:103CC000E26EB5C4E6FFAFC4ADF4B0C4AEF4AF4B22
:103CD000B02BA4AA73D0A3AA71D09CA202D09C98A6
:103CE0009C889CA402D0AACF13F2AACF13F2010E93
:103CF0000101025D02E1FF0E015D05E202011351C7
:103D00000D0A01E038D001C114F402C115F4A4BABF
:103D100001D0FDD70201AACF13F2136B000E0101EF
:103D2000921902E1000E911908E1C80E0125E16E19
:103D3000060E0221E26E13C2E6FF000E921902E1A6
:103D4000010E911908E1A10E0125E16E000E02217C
:103D5000E26E13C2E6FF016B026B914B922B000ED9
:103D6000921902E1020E911905E1AACF13F20201A4
:103D7000136BA39A23D0000E0101921902E1000EE9
:103D8000911908E1C80E0125E16E060E0221E26ECE
:103D900013C2E6FF000E921902E1010E911908E12B
:103DA000A10E0125E16E000E0221E26E13C2E6FFB4
:103DB00001C114F402C115F4014B022B1AC000F02A
:0A3DC0001BC0E1FF1CC0E2FF110070
:103DCA0000C019F001C018F0156ED8CF16F0E0CF78
:103DDA0017F0A0A222D0A1A220D0010E295C006E69
:103DEA00000E2A58016E00C029F001C02AF0150EF3
:103DFA007B6EA00E7A6E800E006E800E2A18005C12
:103E0A0002E12950000807E3010E0601BA6F000E0D
:103E1A00BB6F7990A092A192A1921750E06E1650B2
:103E2A00D86E153A153819C000F018C001F0100004
:103E3A00E6EC2BF00AEC13F0640E296E000E2A6EE3
:103E4A0001018A99930E5D6F010E5E6F936B5F6B32
:103E5A00606B000E605D02E1280E5F5D0AE20E0EE5
:103E6A005F25E16E010E6021E26EE66A5F4B602B10
:103E7A00F0D75F6B606B000E605D02E1800E5F5DE4
:103E8A000AE2930E5F25E16E010E6021E26EE66A98
:103E9A005F4B602BF0D77E86020E7F6E700EB06E7F
:103EAA00AD84DDEC12F00C0E07015B6F6DEC0BF0CC
:103EBA001F0E0B6E710E0C6E1E0E0D6E0D2EFED7A2
:103ECA000C2EFCD70B2EFAD7000001015F6B606B3A
:103EDA00000E605D02E1080E5F5D1CE2030E006EDB
:103EEA00000E016E5FC104F060C105F09CEC04F0A5
:103EFA00600E0024E96E000E0120EA6EEECF3DF757
:103F0A00EECF3EF7EECF3FF734EC0EF001015F4BF8
:103F1A00602BDED748EC10F0D60E07013D6F520E2B
:103F2A003E6F000E3F6F34EC0EF05B0E07013D6FE3
:103F3A00540E3E6F000E3F6F34EC0EF02B0E07014D
:103F4A003D6F500E3E6F000E3F6F34EC0EF0780E50
:103F5A0007013D6F4F0E3E6F000E3F6F34EC0EF0BF
:103F6A00CD0E07013D6F540E3E6F000E3F6F34ECCD
:103F7A000EF07C86020E7D6E700EAB6EA8847DEC10
:103F8A0012F05DC15BF75EC15CF71D0E07015D6F44
:103F9A00540E5E6F000E5F6F7FEC0AF01E0E6E6E9F
:103FAA00B2EC12F00B0E01015D25E16E000E5E21EE
:103FBA00E26E320EE66E5DC13DF75EC13EF7A6ECDB
:103FCA000CF07D0E296E000E2A6E65EC14F0740E4C
:103FDA0001018B6F740E8E6F100E896F770E0701B9
:103FEA003D6F530E3E6F000E3F6F34EC0EF08EC1E4
:103FFA0032F723EC13F000C09FF0000E0001A06F0F
:10400A0048EC10F02E0E07013D6F550E3E6F000E64
:10401A003F6F34EC0EF075EC13F000C09FF001C056
:10402A00A0F00A0E0B6E220E0C6EA10E0D6E0D2E56
:10403A00FED70C2EFCD70B2EFAD729EC12F00A0E5B
:10404A000B6E220E0C6EA10E0D6E0D2EFED70C2ECF
:10405A00FCD70B2EFAD7010E07013D6F000E3E6FFB
:10406A00010E3F6F000E406F0B0E416F560E426FEE
:10407A00000E436F53EC10F0020E07013D6F000E65
:10408A003E6F010E3F6F000E406F6E0E416F550E70
:10409A00426F000E436F53EC10F05C0E0B6E510E24
:1040AA000C6E600E0D6E0D2EFED70C2EFCD70B2E4D
:1040BA00FAD700000D0E5E6E000E5F6EBDEC12F0B8
:1040CA00D20E07013D6F560E3E6F000E3F6F34EC65
:1040DA000EF078EC14F0020E07013D6F000E3E6FF1
:1040EA00010E3F6F000E406F2D0E416F560E426F4C
:1040FA00000E436F53EC10F05C0E0B6E510E0C6EFB
:10410A00600E0D6E0D2EFED70C2EFCD70B2EFAD795
:10411A000000520E07013D6F530E3E6F000E3F6FB7
:10412A0034EC0EF0A00E01018E6FA00E0701326F63
:10413A0023EC13F000C09FF0000E0001A06F070EE1
:10414A000B6E170E0C6E6A0E0D6E0D2EFED70C2E10
:10415A00FCD70B2EFAD7000001018A9D8A99526A70
:10416A000601B66BB76BB86BB96B0401966B976BAC
:10417A0001018F6B906B5F6B606B000E605D02E1FB
:10418A007F0E5F5D0BE2160E5F25E16E040E602165
:10419A00E26E200EE66E5F4B602BEFD7590E0701D9
:1041AA003D6F550E3E6F000E3F6F34EC0EF08FC11F
:1041BA003DF790C13EF70E0E07013F6F010E406FAB
:1041CA00DEEC11F00E0E3D6F010E3E6FA6EC0CF008
:1041DA00880E3D6F570E3E6F000E3F6F34EC0EF0A7
:1041EA0096C43DF797C43EF70E0E07013F6F010EC6
:1041FA00406FDEEC11F00E0E3D6F010E3E6FA6EC25
:10420A000CF048EC10F0790E07013D6F540E3E6F2A
:10421A00000E3F6F34EC0EF08BC18EF1020E0701D7
:10422A005B6F000E5C6F74EC0BF0010E07013D6FC3
:10423A00000E3E6F010E3F6F000E406FD80E416FA9
:10424A00550E426F000E436F53EC10F05C0E0B6E6E
:10425A00510E0C6E600E0D6E0D2EFED70C2EFCD775
:10426A000B2EFAD7000075EC18F09D8AA38AF28CFF
:10427A00F28ED08E0401AB6BAC6B0D0E5E6E000E2F
:10428A005F6E0101036B8A998C98BDEC12F051ECB8
:10429A0018F00D0E5E6E000E5F6E0101936B930EA9
:1042AA005D6F010E5E6F0E6B2E0E0B6EA90E0C6EFD
:1042BA002F0E0D6E0D2EFED70C2EFCD70B2EFAD715
:1042CA00320E296E000E2A6E46EC18F0000E01011D
:1042DA00925D02E1020E915D0BE2000E0601BB192E
:1042EA0002E1010EBA1903E151EC18F001D0EED740
:1042FA007990A0920401A96BAA6B000E0101921990
:10430A0002E1020E9119D8A471D00E0E07015B6F5B
:10431A00010E5C6F900E5D6F570E5E6F000E5F6F41
:10432A007FEC0AF0C80E07013D6F060E3E6F0E0EB7
:10433A003F6F010E406F070E416F11EC11F0000E36
:10434A00011802E1000E001803E19EEC1DF009D0ED
:10435A000701BD0E3D6F530E3E6F000E3F6F34ECEA
:10436A000EF00E0E07015B6F010E5C6F980E5D6F0B
:10437A00570E5E6F000E5F6F7FEC0AF0A10E070109
:10438A003D6F000E3E6F0E0E3F6F010E406F070E1F
:10439A00416F11EC11F0000E011802E1000E001835
:1043AA001CE1F0EC1BF000C02EF001C02FF0000E53
:1043BA00011802E10A0E00180FE137EC19F023EC9C
:1043CA0015F0960E07015B6F000E5C6F6EEC09F03C
:1043DA0000C0A9F401C0AAF409D00701FD0E3D6F7F
:1043EA00530E3E6F000E3F6F34EC0EF051EC18F096
:1043FA00886B81A465D0E60E07013D6F540E3E6FAF
:10440A00000E3F6F34EC0EF0000E81B2010E070170
:10441A005B6F300E5B276DEC0BF0810E07013D6F71
:10442A00550E3E6F000E3F6F34EC0EF0000E010188
:10443A008ABD010E07015B6F300E5B276DEC0BF036
:10444A008A0E07013D6F560E3E6F000E3F6F34EC29
:10445A000EF0000E87B6010E07015B6F300E5B2768
:10446A006DEC0BF0380E07013D6F570E3E6F000ED4
:10447A003F6F34EC0EF00CC15BF76DEC0BF03E0EA7
:10448A0007013D6F560E3E6F000E3F6F34EC0EF083
:10449A00300E522407015B6F6DEC0BF0700E0701B2
:1044AA003D6F570E3E6F000E3F6F34EC0EF0610EFB
:1044BA0007013D6F010E3E6FA6EC0CF048EC10F0C0
:1044CA00930E01015D6F010E5E6F5DC18CF15EC1DD
:1044DA008DF1300E0C5D5F6F606B000E605B800EBD
:1044EA000401AA19006E800E005C02E1040EA95DA7
:1044FA0047E3000E006E01016051005C02E15F516A
:10450A0000083EE25DC15BF75EC15CF7C70E0701BA
:10451A005D6F500E5E6F000E5F6F7FEC0AF0610EEA
:10452A0007015B6F010E5C6F60EC06F000C09FF044
:10453A0001C0A0F0090E01015D2507015B6F000EA5
:10454A0001015E2107015C6F610E5D6F010E5E6FF6
:10455A0000C05FF701C060F7A0EC05F000019F51B1
:10456A0001015D25006E0001A05101015E21016E6D
:10457A00090E0024E16E000E0120E26EE66A0DD0FB
:10458A005DC15BF75EC15CF70D0E07015D6F570EEB
:10459A005E6F000E5F6F7FEC0AF05DC132F75EC19D
:1045AA0033F787EC14F0A2EC14F081A205D00101D4
:1045BA000351000A01E116D001010351010A11E178
:1045CA005250000A0EE10C5100080BE2800E040161
:1045DA00AA19006E800E005C02E1040EA95D01E3D7
:1045EA0001D01DD1780E07013D6F570E3E6F000EA8
:1045FA003F6F34EC0EF08FC13DF790C13EF70E0EBF
:10460A0007013F6F010E406FDEEC11F00E0E3D6F99
:10461A00010E3E6FA6EC0CF0800E3D6F570E3E6FFA
:10462A00000E3F6F34EC0EF096C43DF797C43EF788
:10463A000E0E07013F6F010E406FDEEC11F00E0EF9
:10464A003D6F010E3E6FA6EC0CF0C40E3D6F570E87
:10465A003E6F000E3F6F34EC0EF0040E0B6E0C0E24
:10466A000C6E330E0D6E0D2EFED70C2EFCD70B2EB4
:10467A00FAD70000000001018AB914D081A212D031
:10468A008A8D8D880401966B976B01018F6B906BF5
:10469A000601B66BB76BB86BB96B01018A89526AAE
:1046AA00010E036F9051030802E18F51FE0825E2C3
:1046BA008A9D81A222D00351000A1FE18D98100E13
:1046CA000B6E390E0C6E0D0E0D6E0D2EFED70C2EC6
:1046DA00FCD70B2EFAD7000000008D88100E0B6E47
:1046EA00390E0C6E0D0E0D6E0D2EFED70C2EFCD74C
:1046FA000B2EFAD700000000DCD78AAD90D00C51FF
:10470A003008D8B08CD0800E0401AA19006E800E31
:10471A00005C02E1060EA95DD8A081D0000E9719AF
:10472A0002E1000E961945E18D98000E01019019DB
:10473A0002E1000E8F1929E1160E07015B6F040EC4
:10474A005C6F7D0E5D6F000E5E6F080E5F6F000E70
:10475A00606FA0EC05F004011F6B360E07015B6F5A
:10476A00040E5C6F530E5D6F000E5E6F090E5F6F75
:10477A00000E606FA0EC05F00401406BFF0E07010C
:10478A00326F030E336FADEC14F001015F6B606B97
:10479A00000E605D02E1800E5F5D0BE2160E5F2582
:1047AA00E16E040E6021E26E200EE66E5F4B602B16
:1047BA00EFD7050E026E96C400F097C401F00250BE
:1047CA0005E0003600900136FF0FFAD7160E0024D6
:1047DA0007015B6F040E01205C6F610E5D6F010EB5
:1047EA005E6F200E5F6F000E606FA0EC05F0040193
:1047FA00964B972B000E006E9751005C02E1965182
:10480A0003080DE28FC132F790C133F7ADEC14F013
:10481A0001018F4B902B0401966B976B8D8881A2B7
:10482A0005D001010351020A01E073D001018AADEA
:10483A0066D0DD0E07013D6F530E3E6F000E3F6FCF
:10484A0034EC0EF001018A9D8A998D980401966BC9
:10485A00976BFF0E0701326F030E336FB0EC17F040
:10486A003C0E3D6F540E3E6F000E3F6F34EC0EF05F
:10487A00400E01015F6F000E606F000E605D02E185
:10488A00800E5F5D0BE2160E5F25E16E040E60215D
:10489A00E26E200EE66E5F4B602BEFD7560E0701D5
:1048AA005B6F040E5C6F7D0E5D6F000E5E6F090E0E
:1048BA005F6F000E606FA0EC05F0760E5B6F040E62
:1048CA005C6F530E5D6F000E5E6F0A0E5F6F000E17
:1048DA00606FA0EC05F0FF0E326F030E336FADEC84
:1048EA0014F0750E3D6F520E3E6F000E3F6F34ECA2
:1048FA000EF00401966B976B010E526E0AD08DB8BA
:10490A0002D08C9801D08C888CB802D08D8801D0C6
:10491A008D985250010AD8A483D187A605D00101E7
:10492A000351010801E37CD1480E07013D6F510E86
:10493A003E6F000E3F6F34EC0EF087B601D0FDD704
:10494A003D0E0B6EE10E0C6E3F0E0D6E0D2EFED758
:10495A000C2EFCD70B2EFAD70000000087A605D034
:10496A00020E0101035D01E2F9D7B10E07013D6FA5
:10497A00540E3E6F000E3F6F34EC0EF08FC13DF7C0
:10498A0090C13EF70E0E07013F6F010E406FDEEC3D
:10499A0011F00E0E3D6F010E3E6FA6EC0CF048ECC6
:1049AA0010F0FF0E0701326F030E336FB0EC17F0F1
:1049BA005DC15BF75EC15CF75E0E5D6F570E5E6FA1
:1049CA00000E5F6F7FEC0AF05DC13DF75EC13EF7F6
:1049DA00160E07013F6F040E406FEDEC0BF05DC140
:1049EA003DF75EC13EF72B0E3F6F000E406FEDECB8
:1049FA000BF05DC13DF75EC13EF7360E3F6F040E08
:104A0A00406FEDEC0BF05DC13DF75EC13EF7A6ECE1
:104A1A000CF048EC10F05DC15BF75EC15CF7B00EBC
:104A2A0007015D6F570E5E6F000E5F6F7FEC0AF035
:104A3A005DC13DF75EC13EF7560E07013F6F040E9A
:104A4A00406FEDEC0BF05DC13DF75EC13EF7300EF5
:104A5A003F6F000E406FEDEC0BF00401956B5DC1EA
:104A6A003DF75EC13EF7760E07013F6F040E406FB9
:104A7A00EDEC0BF05DC13DF75EC13EF7A6EC0CF024
:104A8A0048EC10F048EC10F0780E07013D6F4D0E1F
:104A9A003E6F000E3F6F34EC0EF001015F6B606BEE
:104AAA009051605D02E18F515F5D10E25FC132F7A4
:104ABA0060C133F7B0EC17F0160E3D6F040E3E6F6F
:104ACA00A6EC0CF001015F4B602BEAD7860E0701BA
:104ADA003D6F510E3E6F000E3F6F34EC0EF09B0E91
:104AEA0007013D6F530E3E6F000E3F6F34EC0EF020
:104AFA003D0E0B6EE10E0C6E3F0E0D6E0D2EFED7A7
:104B0A000C2EFCD70B2EFAD700000000A70E0701C7
:104B1A003D6F520E3E6F000E3F6F34EC0EF0BDEC4F
:104B2A0012F001018C6B8D6B87A673D00101000E08
:104B3A008D1902E1000E8C196CE18DB802D08C98A7
:104B4A0001D08C888CB802D08D8801D08D981F0E28
:104B5A000B6E710E0C6E1E0E0D6E0D2EFED70C2EE8
:104B6A00FCD70B2EFAD70000000E0401A01902E1AF
:104B7A00010E9F194DE1B60E0701326F040E336F15
:104B8A00330E346F000E356F2BEC17F000C08CF12A
:104B9A0001C08DF1000E026E0150025C02E100506C
:104BAA00000834E26C0E07013D6F560E3E6F000E90
:104BBA003F6F34EC0EF0780E07013D6F4D0E3E6FDD
:104BCA00000E3F6F34EC0EF001015F6B606B905189
:104BDA00605D02E18F515F5D10E25FC132F760C133
:104BEA0033F7B0EC17F0160E3D6F040E3E6FA6ECCD
:104BFA000CF001015F4B602BEAD7860E07013D6F6F
:104C0A00510E3E6F000E3F6F34EC0EF0BDEC12F009
:104C1A008BD7526A0101036B8C6B8D6B51EC18F0C8
:104C2A00000E0401A01902E1010E9F19D8A49CD01C
:104C3A0051EC18F0B60E07013D6F560E3E6F000E8E
:104C4A003F6F34EC0EF0B60E07013D6F040E3E6F57
:104C5A00A6EC0CF048EC10F08BC18EF129EC12F0A6
:104C6A000E0E0701326F010E336FB60E346F040E4B
:104C7A00356F100E366F000E376F6CEC17F0010EA1
:104C8A003D6F000E3E6F010E3F6F000E406FC40E67
:104C9A00416F560E426F000E436F53EC10F0020E36
:104CAA0007013D6F000E3E6F010E3F6F000E406F11
:104CBA000E0E416F010E426F1DEC0CF03D0E0B6E95
:104CCA00E10E0C6E3F0E0D6E0D2EFED70C2EFCD78C
:104CDA000B2EFAD700000000B60E0701326F040E41
:104CEA00336F450E346F000E356F2BEC17F000C092
:104CFA008CF101C08DF1000E026E0150025C02E1DE
:104D0A00005000080CE2170E07013D6F550E3E6F6A
:104D1A00000E3F6F34EC0EF0010E0101036FB60E68
:104D2A000701326F040E336F3B0E346F000E356F7E
:104D3A002BEC17F000C08CF101C08DF1000E026E51
:104D4A000150025C02E1005000080CE2FF0E07016C
:104D5A003D6F540E3E6F000E3F6F34EC0EF0020EA4
:0E4D6A000101036FBDEC12F052EF21F0FFD7F4
:1057CC0010EE1DF0690E006E010E016E0F0EF66EDE
:0E57DC004F0EF76E000EF86EAAEC12F01200DF
:104D78003C3F786D6C2076657273696F6E3D2231A9
:104D88002E302220656E636F64696E673D2255542C
:104D9800462D38223F3E0D3C6B6D6C20786D6C6E55
:104DA800733D22687474703A2F2F7777772E6F705F
:104DB800656E6769732E6E65742F6B6D6C2F322E5E
:104DC80032223E0D3C446F63756D656E743E0D3C3A
:104DD8005374796C652069643D22707572706C65D6
:104DE800506F6C79223E0D3C4C696E655374796C3A
:104DF800653E0D3C636F6C6F723E37666666303099
:104E080066663C2F636F6C6F723E0D3C7769647405
:104E1800683E343C2F77696474683E0D3C2F4C69BA
:104E28006E655374796C653E0D3C506F6C795374A4
:104E3800796C653E0D3C636F6C6F723E376630303F
:104E4800666630303C2F636F6C6F723E0D3C2F509E
:104E58006F6C795374796C653E0D3C2F5374796C83
:104E6800653E0D3C506C6163656D61726B3E3C73D1
:104E780074796C6555726C3E23707572706C6550F0
:104E88006F6C793C2F7374796C6555726C3E0D3C70
:104E98004C696E65537472696E673E0D3C65787433
:104EA800727564653E313C2F657874727564653E31
:104EB8000D3C74657373656C6174653E313C2F7489
:104EC800657373656C6174653E0D3C616C746974DF
:104ED8007564654D6F64653E6175206E69766561C0
:104EE8007520647520736F6C3C2F616C74697475E0
:104EF80064654D6F64653E0D3C636F6F7264696EE7
:074F0800617465733E0D00AA
:024F0F00200080
:024F110020007E
:024F130020007C
:064F1500204964783D0014
:024F1B00640030
:034F1D0020200051
:024F200000008F
:034F22002020004C
:084F2500474554204B4D4C00A0
:0A4F2D00545241434B204F4646000A
:094F3700545241434B204F4E003F
:024F400001006E
:024F420010005D
:014F4400006C
:0B4F450030304830304D303053200039
:024F50000D0052
:104F52003B5200D64F00795000955400005200C3D6
:0B4F620051000353002C53000A5100C3
:024F6D00010041
:094F6F0030312F30312F313600B2
:104F780020626F75746F6E204250323D5248333D47
:104F880030206465206C6120636172746520636CF5
:104F980069636B657220706F75722076616C6964E5
:104FA8006572206C61204361707475726520666952
:104FB8006368696572204B4D4C2067E96E72E92081
:0E4FC80073757220646973706C61790D0A0054
:104FD6002050726F6A6574203A205375727669762E
:104FE6006F725F31384638374A35305F34384D682E
:104FF6007A5F4750535F55424C4F585F374E5F7349
:1050060065756C5F4C4344323131395F3234464307
:10501600313230365F42545F313631302E6D637037
:0550260070690D0A0095
:10502B0020436F6D6D7574617465757220524231DA
:10503B003D313D53746F72655F44617461732073CE
:10504B00757220454570726F6D20206F752043641B
:10505B00652022545241434B204F4E222065742031
:0E506B0022545241434B204F4646220D0A006C
:1050790020536F757263653A20205375727669768D
:105089006F725F31384638374A35305F34384D48AA
:105099007A5F4750535F55424C4F585F374E5F73A5
:1050A90065756C5F4C43445F454570726F6D314D5A
:0E50B900425F42545F3136313132370D0A000A
:1050C70055626C6F78204F4B2C2020202020202009
:1050D70020202020202020202020202020202020C9
:1050E70020202020202020202020202020202020B9
:1050F70020202020202020202020202020202020A9
:0351070020200065
:10510A0020506F7572204170706C692052464F2092
:10511A003A4750535F55626C6F785F504943313854
:10512A00465F5669615F426C7565546F6F74685F5C
:0E513A003136313132372E626173200D0A009A
:10514800507569732C20436C6561722042756666E0
:105158006572207465726D696E616C206469737024
:105168006C617920210D0A20457420617070757971
:0E517800657220737572204250320D0A2000BD
:105186003C2F636F6F7264696E617465733E0D3C8C
:105196002F4C696E65537472696E673E3C2F506C76
:1051A6006163656D61726B3E0D3C2F446F63756D77
:0D51B600656E743E3C2F6B6D6C3E200D004D
:1051C3002055415254312052433720525820203128
:1051D30039323030203C2D2D2070726F6C69666936
:1051E30078203C2D2D2D20636C61766965722054E7
:0D51F30065726D696E616C2050430D0A00FD
:1052000020554152543120524336205458202031E9
:1052100039323030202D2D3E2070726F6C696669F6
:10522000782D2D2D3E204469706C61792054657273
:0B5230006D696E616C2050430D0A0098
:10523B00204469726563746F72793A20433A5C5FFC
:10524B004D696B726F435C5F4D657350726F6A652E
:10525B0074735F4D696B726F435C5F3138463837DF
:0A526B004A35305F4750530D0A002A
:1052750041707075796572207375722042503220C5
:10528500706F757220726563757065726572206CDA
:1052950065206C697374696E67204B4D4C2E2E0D1D
:0252A5000A00FD
:1052A7000D0A0D0A2020417474656E7465204170E3
:1052B70070756920425032206F7520436465202243
:0F52C700474554204B4D4C20220D0A0D0A200064
:1052D600204465636F6461676520646520322054ED
:1052E60072616D6573204E4D45413A202047504707
:0D52F6004741202B204750524D430D0A0028
:1053030020554152543220525820524732203139CD
:1053130032303020203C2D2D204750532055424C15
:095323004F5820374E0D0A2000FE
:10532C0020554152543220545820524731202D2DB3
:10533C002D2D2D3E204D6F64756C652042542048F8
:06534C004330360D0A009B
:1053520020436865636B2070726573656E636520B8
:105362003234464331303236206174204020307866
:0553720041340D0A00AA
:1053770020436865636B2070726573656E63652093
:105387004C43443231313920617420402030783722
:04539700340D0A00C7
:10539B000D0A0D0A20526563757065726572206C7B
:1053AB00652066696368696572204B4D4C20210D41
:0253BB000A00E6
:1053BD0042414420526563657074696F6E206F754C
:1053CD00204465636F6461676520524D430D0A008B
:1053DD000D0A46696E2064652073746F636B616797
:1053ED0065207375722032344643202E2E0D0A002F
:1053FD0042414420526563657074696F6E206F750C
:10540D00204465636F64616765204747410D0A005D
:10541D000D0A20496E69742049324331204861726A
:0F542D006477617265203430304B687A0D0A0065
:10543C005465726D696E6520656372697475726509
:0F544C00207375722032344643202E2E0D0A0035
:10545B0020456E74726565205242323D313D204DC0
:0E546B006F646520426176617264200D0A0054
:10547900200D0A2041726D6520495420554152542E
:0C5489003120262055415254320D0A00FB
:1054950020464F53433D34384D485A2020504C4CFC
:0C54A5002061637469766520200D0A0008
:1054B1000D0A4E756D506167652066696E616C20DD
:0C54C10032344C4331303236203D2000A4
:1054CD00206F7520636F6D6D616E64652022474599
:0954DD0054204B4D4C220D0A0035
:1054E600202052423120696E76657273657572208E
:0954F60053746F7265203D200023
:1054FF000D0A46696E20646520547261636B696E94
:08550F0067204750530D0A000C
:105517000D0A446562757420547261636B696E6726
:07552700204750530D0A005C
:10552E0020496E6974204C43442032313139203287
:06553E007831360D0A0071
:10554400494E49542E4254204843303620424C455B
:0555540055202020009D
:105559002032344C433130323620204E756D506143
:0555690067653D200014
:10556E00203132302078203430203D3E342E3873B6
:03557E0065630062
:105581002020447261706561752053746F72653DAE
:025591002000F8
:1055930041542B4E414D45484330362D3035333938
:0255A3005200B4
:1055A5004C41543A2020202020202020202020205B
:0155B50000F5
:1055B600416C74697475643A2020202020202020D4
:0155C60000E4
:1055C7004C4F4E3A20202020202020202020202031
:0155D70000D3
:1055D80041726D6520496E746572727570747320BE
:0155E80000C2
:1055E90020436865636B20446576696365204020C4
:0155F90000B1
:1055FA0044617465203A2020202020202020202089
:01560A00009F
:10560B00496E69742054696D6572332034306D5363
:01561B00008E
:10561C004E62205361743A202020204669783A204B
:01562C00007D
:10562D00496E6974204144432073757220454131A0
:01563D00006C
:10563E0020205265616479546F577261703D20006D
:0F564E0045746170653A20312073757220340005
:0F565D0045746170653A203220737572203400F5
:0F566C000D5265637570204B4D4C203A0D0A00AE
:0F567B0046696E20696E697420484330362000FE
:0F568A0020204250322053746F7265203D200063
:0F56990045746170653A203320737572203400B8
:0E56A800206973206E6F7420666F756E64004B
:0E56B60055415254312052656375203A200050
:0E56C40055415254312052656375203A200042
:0D56D20020496E697420414443310D0A00E7
:0C56DF002020202020416C74203A200084
:0C56EB002020202048444F50203A20008E
:0B56F70020204820204D2020532000E0
:0B57020020547261636B696E673D000C
:0B570D0055626C6F7820424144200080
:0B571800202020536174656C3A2000D3
:0B57230041542B50494E31323334000A
:0A572E0020666F756E64204F4B007B
:0A573800202047504649583D20004C
:0A574200202020204669783A20005C
:09574C0020204C6174203A200079
:095755004A4A2F4D4D2F4141003D
:09575E004465627574203A2000D4
:0957670032202048415244570051
:0857700020204B4D4C3D2000B0
:0857780050616765203D20002F
:0857800020204964783D20005F
:0857880020496478203D200057
:08579000244750524D432C0048
:085798002447504747412C0053
:0857A000206F6E204932430026
:0857A800204C6F6E203A200036
:0757B00046696E203A20005B
:0757B7004C54433A2020008E
:0657BE0050616765200048
:0357C400202000A2
:0357C7004154004A
:0257CA002C00B1
:020000040001F9
:06FFF800ACF7C5FFF8FFA5
:00000001FF
